:100000000C943E000C9450000C9450000C94500042
:100010000C9450000C9450000C9450000C94500020
:100020000C9450000C9450000C9450000C94500010
:100030000C9450000C9450000C9450000C946F00E1
:100040000C9450000C9450000C9450000C945000F0
:100050000C9450000C9450000C9450000C945000E0
:100060000C9450000C9450000C9450000C945000D0
:100070000C9450000C9450000C94500011241FBE9E
:10008000CFEFCDBFDFE3DEBF28E3A0E0B8E301C0E0
:100090001D92AA30B207E1F70E94C5000C94170127
:1000A0000C9400009091000491FF0AC0811104C0DB
:1000B00082E080930604089582E080930504089509
:1000C0009FB7F894811107C080911104877F8093B6
:1000D00011049FBF0895809111048860F8CF1F928A
:1000E0000F920FB60F9211242F933F934F935F936C
:1000F0006F938F939F93AF93BF93809106389091A6
:100100000738A0910838B0910938409104385091CF
:1001100005389A01205D3C4F283E63E0360728F001
:10012000285E33400196A11DB11D20930438309301
:1001300005388093063890930738A0930838B09319
:1001400009388091003890910138A0910238B0911F
:1001500003380196A11DB11D80930038909301389A
:10016000A0930238B093033881E080938D0ABF9149
:10017000AF919F918F916F915F914F913F912F918F
:100180000F900FBE0F901F90189588ED90E084BFE0
:100190009093610083E5809302068EE080930506CC
:1001A00090E29093030680910006816080930006A0
:1001B00021E02093030A8EEF8093260A8093270A7A
:1001C00080E88093280A80932A0A80932C0A8093DF
:1001D000290A80932B0A80932D0A3BE03093000A72
:1001E0004DEF51E04093AE0A5093AF0A20938C0A32
:1001F0001092810A8093820A81E18093800A789428
:1002000082E0809301042FB7F894909302048091C8
:100210001504877F809315042FBF8091080485FD06
:1002200004C080E00E945200F8CF81E0FBCFF89438
:02023000FFCFFE
:00000001FF
